:1000000012C0189518951895189518951895189563
:100010001895189518951895189518951895189578
:100020001895189518958FED8DBFC0ECE0EC4E2E0D
:10003000DD275D2EEEE7F0E0A0E6B0E0A89584B7FE
:10004000082E877F84BF88E1992781BD91BD8827CD
:100050008D933197E9F7ABD266248FE087BB80E0C0
:1000600088BB8FEF81BB80E082BB84E690E013D336
:100070008CE0E5D2BF98A7E69C9197FF04C0B799A2
:100080000EC09F779C93B79B0AC088E29F939927E5
:1000900002D39F91B79B03C090689C9317D26DD2F7
:1000A000ECE0F7E062D267D2ECE1F7E05ED2E2E0AA
:1000B000F0E074D280E080936400A1E6FFD280E09B
:1000C0008093630080E08093650057D2ECE2F7E014
:1000D0004CD288E087BB80E788BB8AE090E0DBD227
:1000E00081E080936000A6E30C9105FB81E00EF4B3
:1000F00080E08F93A6E30C9106FB81E00EF480E094
:100100009F918923882309F401C00CD182E0809358
:100110006000A6E30C9104FB81E00EF480E08F9375
:10012000A6E30C9105FB81E00EF480E09F9189230A
:10013000882309F401C0F6D083E080936000A6E331
:100140000C9104FB81E00EF480E08F93A6E30C9108
:1001500006FB81E00EF480E09F918923882309F457
:1001600001C0E0D080E187BB88E688BB8AE090E0F0
:1001700092D284E080936000A6E30C9105FB81E0BD
:100180000EF480E08F93A6E30C9106FB81E00EF461
:1001900080E09F918923882309F401C0C3D085E0C2
:1001A00080936000A6E30C9105FB81E00EF480E0F3
:1001B0008F93A6E30C9106FB81E00EF080E09F9107
:1001C0008923882309F401C0ADD086E080936000C4
:1001D000A6E30C9105FB81E00EF080E08F93A6E38F
:1001E0000C9106FB81E00EF480E09F918923882327
:1001F00009F401C097D080E287BB88E588BB8AE01C
:1002000090E049D287E080936000A6E30C9104FB64
:1002100081E00EF080E08F93A6E30C9106FB81E075
:100220000EF480E09F918923882309F401C07AD0DD
:1002300088E080936000A6E30C9104FB81E00EF45B
:1002400080E08F93A6E30C9106FB81E00EF080E046
:100250009F918923882309F401C064D089E08093A9
:100260006000A6E30C9104FB81E00EF480E08F9324
:10027000A6E30C9106FB81E00EF480E09F918923B8
:10028000882309F401C04ED080E487BB88E388BB93
:100290008AE090E000D28BE080936000A6E30C91AE
:1002A00004FB81E00EF080E08F93A6E30C9105FB48
:1002B00081E00EF480E09F918923882309F401C036
:1002C00031D08AE080936000A6E30C9104FB81E0CA
:1002D0000EF480E08F93A6E30C9105FB81E00EF411
:1002E00080E09F918923882309F401C01BD08CE012
:1002F00080936000A6E30C9104FB81E00EF480E0A3
:100300008F93A6E30C9105FB81E00EF080E09F91B6
:100310008923882309F401C005D08AE090E0BBD18D
:10032000D8CEA3CE939A84E690E0B5D1939884E694
:1003300090E0B1D100916400013009F001C02AC001
:1003400000916400023009F001C047C000916000D4
:100350000B3009F00CC011D1EAE3F7E006D1A4E6B6
:100360008C918F5F8C9380E080936300B2CE00917C
:1003700060000C3009F00DC0EAE0F0E0A4E1BED16D
:10038000A1E60D911C910417150709F001C088C062
:1003900065C036C0009160000C3009F01DC0EAE075
:1003A000F0E0A4E1ABD1A1E60D911C910417150773
:1003B00009F401C053C0A1E681D180E080936300BD
:1003C00080E080936500A4E68C918F5F8C93D5D0FC
:1003D000EAE4F7E0CAD07DCE13C0009160000C3093
:1003E00009F00EC0EAE0F0E0A1E67BE776D1C5D0E7
:1003F000EAE5F7E0BAD043D0E2E0F0E0CFD05ACE61
:10040000A3E68C918F5F8C930091630046E0040F0C
:10041000A5E60C938FEBA5E61C91BED0EAE6F7E0CB
:10042000A4D000916300043010F009F001C001C0B5
:1004300015C0A1E60D911C914AE050E083D0A1E6E1
:100440000D931C93A1E60D911C91A0E64D915527AB
:10045000040F151FA1E60D931C9308958ED0ECE6B2
:10046000F7E083D0939AE3E0F0E098D0939883D0BC
:10047000ECE0F7E07AD0E4E1F0E090D01BCE84E647
:1004800090E009D1939A88EC90E005D1939888EC9C
:1004900090E001D1939A88EC90E0FDD09398089574
:1004A0006CD0EAE5F7E061D0EADF65D0EAE7F7E093
:1004B0005CD08CE291E0EFD0949AE1E0F0E06ED075
:1004C00094985BD0E1E0F0E069D0F4CDE1E0F0E0B9
:1004D00065D0B79901C014C0EAE0F0E002ED14E085
:1004E000A0E1BB277BE7F9D0CADF47D0E8E8F7E017
:1004F0003CD041D0E8E9F7E038D0E4E0F0E04ED07D
:10050000089504D01FD000FC0CD008950024E89476
:1005100057FF02C009D0689400F80BD010F80124EE
:10052000089502D009D00895509540954F5F5F4FD0
:100530000895E89417FF0895009510950F5F1F4FD9
:1005400068940895752F642F55274427FF93F1E190
:10055000889405C010F4460F571F56954795179578
:100560000795FA95B9F7FF910895A4D0802D11F061
:1005700060D0FBCF089580EC62C081E060D014D0E1
:1005800080E85DC08FE7213039F08FEB223021F019
:100590008FE8233009F08FEC810F51C088EE93E093
:1005A0007AD03197D9F7089583E0992774C08AEFFC
:1005B00090E071D0BB9ABA9AB99AB89A8E9A8D9AED
:1005C000959885E090E067D09698C398C298C19AB4
:1005D000C09A969AEF93FF93E5E1F0E050D0FF9137
:1005E000EF91969855D0969AEF93FF93E5E1F0E05E
:1005F00046D0FF91EF9196984BD0969AEF93FF9348
:10060000E5E1F0E03CD0FF91EF91969841D0C098A1
:10061000969AEF93FF93E5E1F0E031D0FF91EF91EF
:10062000969836D088E20BD08EE009D086E007D0CD
:100630000895959A829505D004D02AD0089595986A
:10064000F9CF859510F4C09A01C0C098859510F433
:10065000C19A01C0C198859510F4C29A01C0C29890
:10066000859510F4C39A01C0C398969AEF93FF93AF
:10067000E5E1F0E004D0FF91EF919698089531976D
:10068000F1F70895689462F80895E89462F808957F
:1006900081E090E000C0EF93FF93EE27E82BE92B79
:1006A00031F0EAEFF0E03197F1F70197D1F7FF91E0
:1006B000EF910895C89531960020089582E001C019
:1006C00084E099279D938A95E9F70895E199FECFF3
:1006D000EEBB3196089591E001C092E07B3751F472
:1006E0007FB7F894F3DF8D918DBBE29AE19A9A95EA
:1006F000C9F77FBF7727089591E001C092E0E6DF58
:10070000E09A8DB38D939A95D1F708955757572E48
:100710004156522E344D472E434F4D00436F646572
:100720004C6F636B415652202D20520020202045F3
:100730006E74657220636F64650020456E74657227
:10074000206F6C6420636F64650020456E74657271
:10075000206E657720636F64650020436F646520B9
:10076000616363657074656400002A002020204383
:100770006F64652077726F6E670020202020556EB1
:100780006C6F636B656400002020496E6974696159
:100790006C20636F64650000202020202069732096
:0807A000202031323334000047
:00000001FF
